:100000000C94F0000C940D010C940D010C94060559
:100010000C940D010C940D010C940D010C940D0128
:100020000C940D010C943A010C940D010C940D01EB
:100030000C940D010C940D010C940D010C940D0108
:100040000C940D010C94D0080C940D010C94C8076D
:100050000C940D01FF008C80A803AC02CC01800C35
:100060008179820083008400800881F5820083000A
:100070008400800D81AD820283008400800981D5D7
:10008000820383168400800D81DB8202830084005A
:10009000800981CD82A183018400800D81DF8202ED
:1000A00083008400800981CE820383168400800D42
:1000B00081B7820383008400800981CE825183014D
:1000C0008400800D81C2820383008400800981CE78
:1000D000825183048400800D81C9820383008400DF
:1000E000800981CF82A183048400800D81CC8203AA
:1000F00083008400800981D082A183048400800D64
:1001000081CE820383008400800981CD8201830433
:100110008400810E825F83A1840081D1825183A4F7
:10012000840081D182518301840081F0821183088F
:10013000840081C182018304840081E082028316ED
:1001400084008194820F8301840081038200830BE9
:100150008400810082A08345840081D182A18344F0
:10016000840081CD82A18344840081AE8202831603
:100170008400800D8135820783008400800981001E
:1001800082FF83A5840E8100827F83A9840381007E
:1001900082FF835284078100823F837E844C8100EA
:1001A00082F083028400810082ED83368400810026
:1001B00082B483DB840081008255835584058100ED
:1001C000824483448400810082FE83FF843F810057
:1001D00082C8838F8409810082118300840080009B
:1001E00011241FBECFE5D4E0DEBFCDBF11E0A0E6F5
:1001F000B0E0ECEEF9E202C005900D92A63DB10729
:10020000D9F713E0A6EDB1E001C01D92A63CB107FD
:10021000E1F70E941E070C94F4140C940000582F70
:10022000DB01282F392FF90102C0919311968E2FEF
:10023000851B9C919923C9F70895DC019091610079
:10024000FD0186E58193892F82958F70805D1196DF
:100250008C938EE281839F70905D928384E00895F9
:1002600080E683BF12BE89B7816089BF83B784608F
:1002700083BF08951F920F920FB60F9211240F9013
:100280000FBE0F901F90189514BC8BE483BD89B7E7
:10029000806889BF12BC85B58F6085BD0895DF93E6
:1002A000CF9300D0CDB7DEB71A82198205C08981FD
:1002B0009A8101969A83898389819A81845F91408A
:1002C000B0F31A82198205C089819A8101969A83B6
:1002D000898389819A81845F9140B0F31A8219825F
:1002E00005C089819A8101969A83898389819A813F
:1002F000845F9140B0F30F900F90CF91DF910895FC
:10030000843029F48091410384608093410380E02C
:100310000895CF93DF93EB01863010F08FEF11C07B
:10032000E82FF0E0EE0FFF1FEA55FE4FA081B181EC
:1003300013968C9188830190F081E02D84858983C8
:1003400082E0DF91CF910895E82FF0E0EE0FFF1FDC
:10035000EA55FE4F0190F081E02D84850895E2E496
:10036000F3E0E80FF11D80810895CF93DF93A82F6C
:10037000EB01863010F08FEF25C08FE38883B0E06B
:10038000AA0FBB1FAA55BE4FED91FC91119781A5F5
:100390008983ED91FC91119780A58A83ED91FC9161
:1003A000119787A18B83ED91FC91119786A18C8386
:1003B000ED91FC91119785A18D83ED91FC9184A124
:1003C0008E8387E0DF91CF910895982FDA0160FF47
:1003D0000BC0E82FF0E0EE0FFF1FEA55FE4F019033
:1003E000F081E02D8C9181A761FF0DC0E92FF0E035
:1003F000EE0FFF1FEA55FE4F0190F081E02D1196A0
:100400008C91119780A762FF0DC0E92FF0E0EE0FED
:10041000FF1FEA55FE4F0190F081E02D12968C915E
:10042000129787A363FF0DC0E92FF0E0EE0FFF1FC7
:10043000EA55FE4F0190F081E02D13968C911397B1
:1004400086A364FF0DC0E92FF0E0EE0FFF1FEA5511
:10045000FE4F0190F081E02D14968C91149785A3A6
:1004600065FF0CC0E92FF0E0EE0FFF1FEA55FE4FCD
:100470000190F081E02D15968C9184A380E0089581
:10048000E82FF0E0E45BFC4FE081E330A1F0E430E2
:1004900028F4E13051F0E23051F40BC0E63079F04D
:1004A000E73079F0E53019F408C087E0089580E07E
:1004B000089583E0089581E0089588E0089588E133
:1004C000089588E308958FEF90E0089584ED0895EE
:1004D000823010F08FEF0895A82FB0E0FD01E65BA9
:1004E000FC4F6083FD01E85BFC4F4083FD01E65C4F
:1004F000FD4F8FEF8083A55DBD4F4C9380E0089545
:10050000CF93DF93982FEB01823010F08FEF1AC05A
:1005100082E0888319821A82992309F481E08B830F
:10052000E92FF0E0DF01A65BBC4F8C918C83E85B88
:10053000FC4F80818D83992311F082E001C081E01E
:100540008E8387E0DF91CF910895FC0181E0808365
:1005500082E081830895FB01823010F08FEF0895CF
:10056000882319F0813061F404C082E0808381E047
:1005700003C084E0808382E08183828383E00895E6
:1005800010821182128283E0089580E00895FB01B9
:10059000882311F08FEF089580916200808380910D
:1005A0006300818382E0089580E00895CF93DF9314
:1005B000FB01EA01823051F0833018F4813051F4AC
:1005C0000BC08B30B1F08C3029F40CC0808161817C
:1005D0000E94570A80E01AC080810E94300A8883F6
:1005E00081E014C06E5F7F4F808141810E94380B93
:1005F0000DC080818883BA016E5F7F4F8081418109
:100600000E94830A89838F3F09F08E5FDF91CF912B
:100610000895FF920F931F93CF93DF93F82EEB0172
:10062000142F0FB7F8940E940208882311F40E9437
:10063000AC080FBF219611508F2DBE01412F0E9493
:100640001A08DF91CF911F910F91FF9008951F938A
:10065000CF93DF93162FC82FD0E0DE01A45BBC4FF1
:100660008C91843009F499C0853048F4823069F166
:10067000833008F05EC0813009F046C10AC0863080
:1006800009F4F3C0863008F4B8C0873009F03CC1E3
:100690001FC1FE01EE0FFF1FEA55FE4F0190F081D2
:1006A000E02D262F30E047A1C25DDD4F888190E02C
:1006B000840F911D281739070CF426C182E08C9312
:1006C00080916000678145E01DC1FE01EE0FFF1FB4
:1006D000EA55FE4F0190F081E02D87A1861740F08A
:1006E00081E08C9380916000678144E00E94141047
:1006F000FE01EE0FFF1FEA55FE4FA081B181212FB1
:1007000030E098964C919897FE01E25DFD4F808114
:1007100090E0840F911D821793070CF0F5C0C45B25
:10072000DC4F83E088838091600017966C9143E0F2
:10073000E9C0FE01EE0FFF1FEA55FE4F0190F08168
:10074000E02D80A5861740F082E08C9380916000B8
:10075000678142E00E941410FE01EE0FFF1FEA5570
:10076000FE4FA081B181212F30E099964C9199974D
:10077000FE01E25DFD4F808190E0840F911D8217A4
:1007800093070CF0C1C0C45BDC4F84E08883809188
:10079000600017966C9141E063C0FE01EE0FFF1FF1
:1007A000EA55FE4F0190F081E02D81A5861758F0A3
:1007B00083E08C9380916000678140E00E94141078
:1007C0008FEF80934B03FE01EE0FFF1FEA55FE4FA4
:1007D0000190F081E02D86A1181708F495C0C45B44
:1007E000DC4F85E0888380916000678147E00E944C
:1007F00014108FEF80934B0387C0FE01EE0FFF1F95
:10080000EA55FE4F0190F081E02D85A1681740F078
:1008100086E08C9380916000678149E00E9414100B
:10082000FE01EE0FFF1FEA55FE4FA081B181412F5F
:1008300050E096968C91969790E0FE01E25DFD4F18
:100840002081821B9109481759070CF05DC0C45BD9
:10085000DC4F84E088838091600017966C9146E0BD
:100860000E94141010924B034FC0FE01EE0FFF1FA9
:10087000EA55FE4F0190F081E02D84A1681740F009
:1008800087E08C938091600067814BE00E94141098
:10089000FE01EE0FFF1FEA55FE4FA081B181412FEF
:1008A00050E095968C91959790E0FE01E25DFD4FAA
:1008B0002081821B91094817590734F5C45BDC4F2E
:1008C00085E088838091600017966C9148E01AC09B
:1008D000FE01EE0FFF1FEA55FE4F0190F081E02D63
:1008E000462F50E084A190E0C25DDD4F2881821B3D
:1008F00091094817590744F486E08C938091600071
:1009000067814AE00E941410DF91CF911F910895F2
:10091000DF93CF9300D00F92CDB7DEB7E82FF0E092
:10092000EC5CFD4F80818169898380E0BE016F5F4F
:100930007F4F42E00E946E13823011F08FEF02C0B1
:100940009981892F0F900F900F90CF91DF9108958B
:1009500083FF5BC00E940010882309F056C090916D
:10096000D801E92FF0E0E45CFD4F8081813099F4FB
:10097000892F0E948804682F882369F09091D801FC
:10098000E92FF0E0EE5BFC4F8081861721F0608359
:10099000892F0E9427038091D8018F5F8093D8010F
:1009A000863010F01092D8018091D901813081F009
:1009B000813028F08230A9F0833039F51DC085B12F
:1009C0008093470383EE87B987EC86B981E011C035
:1009D00085B18093440382EE87B987EC86B982E0C3
:1009E00008C085B18093450381EE87B987EC86B94D
:1009F00083E08093D901089585B18093460380EE0A
:100A000087B987EC86B91092D90108951F920F9289
:100A10000FB60F9211242F933F934F935F936F93D1
:100A20007F938F939F93AF93BF93EF93FF938091A7
:100A3000D6018F5F8093D601843639F480914103CB
:100A40008860809341031092D6018091DA01882357
:100A500039F081508093DA01882311F40E94240A2E
:100A6000FF91EF91BF91AF919F918F917F916F9186
:100A70005F914F913F912F910F900FBE0F901F905C
:100A80001895EF92FF920F931F93DF93CF9300D0AF
:100A900000D0CDB7DEB78C0188E090E07E010894ED
:100AA000E11CF11CB70144E00E94AD14F80182E59D
:100AB000819385E6D80111968C9311978CE68183FA
:100AC0008AE3828392E09701F901E90FF11D8081A9
:100AD00082958F70805D14968C93149780818F70AF
:100AE000805D15968C931597915012969F3F61F7F4
:100AF0008AE00F900F900F900F90CF91DF911F9190
:100B00000F91FF90EF9008958F929F92BF92CF9296
:100B1000DF92EF92FF920F931F93DF93CF9300D05A
:100B200000D0CDB7DEB74C0184E090E08E010F5FBE
:100B30001F4FB80144E00E94AD1433E0CC24DD2403
:100B40007601A801BE2DAD2D9C2D8827FA01E30F5B
:100B5000F11D2081C22EDD24EE24FF24C82AD92ACB
:100B6000EA2AFB2A315070F7BB2484010B0D111DBA
:100B7000C701B6012AE030E040E050E00E94D21404
:100B8000605DF8016083B394C701B6012AE030E0EC
:100B900040E050E00E94D214C901DA016C017D01ED
:100BA000C114D104E104F10401F73B2D3695D401C1
:100BB000EB2DF0E03197E80DF91D20E006C09C9187
:100BC00080818D9390832F5F31972317C0F38B2DF6
:100BD0000F900F900F900F90CF91DF911F910F9179
:100BE000FF90EF90DF90CF90BF909F908F900895EF
:100BF0009F92AF92BF92CF92DF92EF92FF920F93AC
:100C00001F93CF93DF93E2E4F2E0119283E0E134AB
:100C1000F807D9F781E080934202809346028093DF
:100C20004A0210924B0210924C02E8EBF1E0AEE463
:100C3000B2E080E003C09D9331968F5F908199234D
:100C4000D1F790E0282F206C20934D02BC016C5FFF
:100C50007F4FEC012C96815B9D4FDC01EAECF1E0CB
:100C600002C04D9331962A2F281B40814423C9F797
:100C700030E0CE5BDD4F822F806C8883AB014F5F0D
:100C80005F4F420F531FEA012896BA01655B7D4F03
:100C9000DB01EEECF1E002C08D9331962A2F261B8A
:100CA00080818823C9F730E0CE5BDD4F822F806CD6
:100CB0008883CA010196820F931FDC01A55BBD4F9B
:100CC00030916100FD0126E52193232F22952F709D
:100CD000205D11962C932EE221833F70305D32838C
:100CE000FC01E65BFD4F24EC2083A5E0EA2EF12C0D
:100CF000E80EF91E8C01035F1F4F805B9D4F0E9421
:100D0000840590E00E5B1D4F282F206CF801208396
:100D100001968E0D9F1DFC01EE5BFD4F20EC2087A0
:100D20007C010894E11CF11C8C01075F1F4F845B60
:100D30009D4F0E94410590E00E5B1D4F282F206CB7
:100D4000F801208301968E0D9F1DFC01EE5BFD4F87
:100D500021EC2087EC012196FC01E55BFD4F02C0F0
:100D60001192E901CE01877090709E012F5F3F4F75
:100D70000797B1F7F3E035952795FA95E1F72093BA
:100D80004B028AE492E06C2F0E94890CFE01EE5B1C
:100D9000FD4F8087E9E0CE2ED12CCC0EDD1EC601A2
:100DA00073E0959587957A95E1F780934702EE2455
:100DB000FF245601F701E556FE4F91806281C62F50
:100DC000D0E0D501AE0DBF1DAE5BBD4F20E030E0E1
:100DD000AE014C5F5F4F04C081918D932F5F3F4FF9
:100DE00042175307CCF787010C0D1D1DC801895B05
:100DF0009D4F0E94890C0E5B1D4FF8018383C80133
:100E000064E00E94890CF801848397FC04C0259655
:100E1000EC0EFD1ECFCF82E492E067E00E94890CC9
:100E200080934902DF91CF911F910F91FF90EF9036
:100E3000DF90CF90BF90AF909F9008951F93CF9376
:100E4000DF930E944F010E944F010E944F010E94B8
:100E50004F010E944F011092D6018CE08093430312
:100E600082E980933502C6EAD1E0ACE3B2E020E04B
:100E700030E044E092E0E881F98183818150823062
:100E800018F484858C9301C01C92F901E45BFC4F3B
:100E90004083F901E25DFD4F90832F5F3F4F229623
:100EA00011962630310539F780B7826080BF80EF18
:100EB0008BBB80E48ABB9FEF98BB88E087BB95BB68
:100EC00014BA92BB11BA0E944F01809160000E9437
:100ED000DC0780E00E94C51214BC8BE483BD89B797
:100EE000806889BF12BC85B58F6085BD8091600028
:100EF0000E94A50C0E94890D789410922D0203C0C7
:100F000016BE0E944F010E9477088823C9F70E94ED
:100F1000270A0E944F011FEF04C00E944F01115089
:100F200011F09D9BFACF81E00E94300A809361000E
:100F30000E94F80510922D0203C016BE0E944F01B8
:100F40000E9477088823C9F790914103992341F0C3
:100F50008FB7F894109241038FBF892F0E94A80485
:100F600086E693E060E20E94B108682F882321F0B2
:100F700086E693E00E94940D0E947708E5CF80E713
:100F80008CBF88E083BF89B7826089BF12BE089595
:100F90001F920F920FB60F9211248F9313BE809160
:100FA00022028F70813011F480E886BF8F910F90FC
:100FB0000FBE0F901F9018958093DC0110921F02B6
:100FC00010922002109221021092220290E290B917
:100FD000816082B98FEF83B980E78CBF88E083BFDF
:100FE00089B7826089BF12BE84E886BF089580E811
:100FF00086BF10921F0210922002109221021092BE
:101000002202089580912202089584E690E00DC0A6
:10101000019711F481E0089524E605C00000000066
:101020000000000000002150C8F706B600FCF0CF19
:1010300080E008950F931F93CF93DF93082FEB0168
:10104000142F8AE08093DA010E940508882311F0AA
:1010500080E886BF81E0809322020093FE018093A6
:1010600021021F5F10932002115000FF0BC00CC023
:101070001150E12FF0E0DE01AE0FBF1F8C91E45262
:10108000FE4F83A31123A1F780E886BF90916000F3
:101090009F719F5F08C0000000000000000000007A
:1010A0008150C8F701C0292F215011F088E2F8CFF4
:1010B0009F5F83B383708330B1F782E005C0000087
:1010C00000000000000000008150C8F783B3837067
:1010D000833049F785E08093DA0185EA86BF12BE46
:1010E0008CE083BFDF91CF911F910F910895DF9323
:1010F000CF930F92CDB7DEB783B38370833041F0C7
:101100008091DA01882319F585E08093DA011FC008
:101110001092DA0106B600FC1AC080911F028823E3
:10112000B1F4198203C089818F5F898389818431F9
:10113000D0F380E886BF83E08093220210921F02E2
:1011400085EC86BF85E08093DA0180E001C081E014
:101150000F90CF91DF91089580E886BF1092DA0159
:1011600008959C0190911F02992311F460E016C02C
:101170001092DA01961708F4692FEDEDF1E0D9012C
:10118000262F30E02E0F3F1F02C081918D93E21772
:10119000F307D9F71092220210921F02862F0895AA
:1011A0001F920F920FB60F9211242F933F938F939C
:1011B0009F93EF93FF9381B1887F883609F4F0C045
:1011C00020912D02893658F5803309F477C0813398
:1011D00098F4883109F45BC0893138F4883009F417
:1011E0004CC0803109F01AC148C0803209F466C091
:1011F000883209F013C14BC0803509F47AC08135BB
:1012000038F4883309F461C0803409F007C162C042
:10121000883509F486C0803609F000C192C088394B
:1012200009F4BEC0893998F4803809F497C0813830
:1012300038F4803709F485C0883709F0EFC0B0C0B2
:10124000883809F4ADC0803909F0E8C087C0803B18
:1012500009F4DBC0813B38F4803A09F4B0C0883A25
:1012600009F0DCC0B9C0803C09F4CFC0883C09F467
:10127000CCC0883B09F0D2C0B7C085E08093DA01CA
:1012800080912D02806880932D021092210280911E
:101290002D02816880932D0290912102809120027D
:1012A000981750F4E92FF0E0E452FE4F82A183B981
:1012B0009F5F9093210233C084E9ADC080912D02DD
:1012C000826880932D0284E9ADC0246820932D02AA
:1012D00085EAA8C0286820932D021092210284E09C
:1012E0008093220280911F028230C8F085EC86BF75
:1012F0009FC0206920932D022091210283B1E22F0B
:10130000F0E0E452FE4F81832F5F2093210230E012
:1013100080911F0290E00197281739073CF385E878
:10132000E6CF206A20932D028091210293B1E82F0D
:10133000F0E0E452FE4F91838F5F8093210284E9B5
:1013400048C0216020932D0283B18093DD0181E0AC
:101350008093210285EC86BF84E068C090912102D1
:1013600083B1E92FF0E0E452FE4F81839F5F9093B9
:10137000210284E08093220220912D029F3120F4EB
:10138000226020932D02B2CF206820932D0285E0A9
:101390008093220290931F021092210284E8A7CF2B
:1013A00080912D02846080932D0280912102809390
:1013B0001F021092210284E886BF85E837C02860AA
:1013C00020932D028091210280931F02109221020E
:1013D00084E886BF85E02AC0206120932D02109208
:1013E000210281E08093220280912D02806280930D
:1013F0002D0290912102E92FF0E0E452FE4F82A1EC
:1014000083B99F5F9093210271CF80912D028064F8
:1014100080932D0284E886BF82E008C0206C209370
:101420002D0284E886BF8091220280688093220288
:1014300012BEFF91EF919F918F913F912F910F904D
:101440000FBE0F901F90189580E886BF089588B34F
:10145000836088BBC29887B3876087BB11BA089541
:10146000982F882311F490EF20C0823011F490E17E
:101470001CC08FEF81BB92BBC29A00000000C298D3
:1014800011BAC1980000000000000000000028E828
:1014900033E104C0019720E030E09E9BC901009732
:1014A000C9F790B3C19A8FEF82BB892F0895E82FB7
:1014B0008C57843060F4F0E0EA51FD4F60838091F6
:1014C000620380FF02C0DE980895DE9A08958FEFD0
:1014D00081BBE2BBC29A00000000C29862BBC09808
:1014E0000000000000000000000028E833E104C014
:1014F000019720E030E09E9BC9010097C9F7C09A90
:101500008FEF82BB0895EF92FF920F931F93CF93BB
:10151000DF93162FF72EE42E80E40E94300A082F66
:10152000212F3F2DC901EC0110E0FF2436C080E5DA
:1015300060E10E94570A04C0F39488ECF816A9F100
:1015400080E50E94300A80FDF7CF84E50E94300AD2
:1015500088830F3F31F00F5F80E4602F0E94570AAD
:101560001AC084E40E94300A682F8F3F19F06F5F21
:1015700084E40AC084E460E00E94570A88E40E9480
:10158000300A682F6F5F88E40E94570A80E460E0A9
:101590000E94570A00E01F5F21961E1540F211318C
:1015A00020F4E11610F0812F01C08FEFDF91CF9171
:1015B0001F910F91FF90EF900895CF93DF9383E6F3
:1015C00063E00E94570AC4E5D0E0FE0184912196B1
:1015D000FE0164910E94570A2196F1E0C03EDF07A8
:1015E000A1F783E660E00E94570A85EB60E80E945D
:1015F000570A88EB6FE90E94570A89EB68E80E9456
:10160000570A8FEC60E40E94570A80EE6FE30E9455
:10161000570A81EE64E60E94570A82EE6AE30E944E
:10162000570A83EE65EC0E94570A84EE6AE00E9436
:10163000570A85EE61E00E94570A87EB6FE10E942E
:10164000570A88E961E20E94570A89E963E40E9427
:10165000570A84EB6BEC0E94570A82EB60E30E940E
:10166000570A88EC60E40E94570ADF91CF910895F1
:10167000DF92EF92FF920F931F93DF93CF9300D0EF
:1016800000D000D0CDB7DEB7FB01D42E8823E9F41B
:101690008B01EE24FF2416C08CE4F80160810E94C7
:1016A000570A80E560E80E94570A04C0F394F8ECFA
:1016B000FF1621F180E50E94300A80FDF7CFE39408
:1016C0000F5F1F4FED1440F31BC08130C9F484E05D
:1016D0004817A1F484E989834A8380818B838181BF
:1016E0008C8382818D8383818E8380E0BE016F5FD6
:1016F0007F4F46E00E943613863011F08FEF01C015
:1017000080E026960FB6F894DEBF0FBECDBFCF9116
:10171000DF911F910F91FF90EF90DF90089584ED7E
:10172000809352031092530388E0809354038DE713
:10173000809355031092560310925703109258034A
:101740001092590310925A0380EC80935B0381E05E
:1017500080935C0380E062E573E04BE00E94361307
:10176000AF9808958CED809352031092530387E055
:1017700080935403109255038BE980935603109283
:101780005703109258031092590388E080935A032C
:1017900081E080935B0380E062E573E04AE00E94B1
:1017A000361308951F93182F8C3010F08FEF3AC026
:1017B0008650843010F492E001C091E084ED809373
:1017C00052039093530385ED8093540380E062E5C8
:1017D00073E043E022E00E94BE13163050F481E033
:1017E00090E002C0880F991F1A95E2F79091530379
:1017F00015C040915303812F90E01A3018F021E179
:1018000030E002C029E030E0281B390B81E090E095
:1018100002C0880F991F2A95E2F7942F9823892FE9
:1018200009F081E01F910895FF920F931F93182FE5
:10183000F62E8C3010F08FEF68C08650843010F494
:1018400002E001C001E084ED809352030093530352
:1018500085ED8093540380E062E573E043E022E08D
:101860000E94BE1340915303FF2001F5163040F44F
:1018700081E090E002C0880F991F1A95E2F712C02C
:10188000812F90E01A3018F021E130E002C029E009
:1018900030E0281B390B81E090E002C0880F991FCF
:1018A0002A95E2F7982F909594231EC0163040F4A5
:1018B00081E090E002C0880F991F1A95E2F712C0EC
:1018C000812F90E01A3018F021E130E002C029E0C9
:1018D00030E0281B390B81E090E002C0880F991F8F
:1018E0002A95E2F7942F982B84ED8093520300936E
:1018F000530381E0809354039093550380E062E5A5
:1019000073E044E00E94361380E01F910F91FF9036
:101910000895AC0120E006C06150FA01E60FF11D08
:101920008081280F6623C1F7822F81950895DC01FD
:1019300020E006C06150FD01E60FF11D8081280FF7
:101940006623C1F7842F820F0895CF93DF93682F0A
:1019500090E08057904095958795482F4066C6EA5D
:10196000D1E020E030E0522FA881B981F901EE5496
:10197000FE4F8081855014968C93149713969C91FA
:101980001397892F8150823048F418968C911897BC
:10199000813C71F419964C9319970AC0923141F425
:1019A0001C968C911C97813C19F41D964C931D97A5
:1019B0005C9311961C92119715966C932F5F3F4F75
:1019C00022962630310579F6DF91CF910895DC011A
:1019D00011968C9111979C91890F819512969C91EB
:1019E0001297981719F02FEF3FEF19C0262F2150AB
:1019F000FD01E60FF11D3197608190E006C0215096
:101A0000FD01E20FF11D8081980F2223C1F791950E
:101A1000691719F420E030E002C02EEF3FEFC90152
:101A20000895CF92EF920F93FC014083EE0CEE0CE1
:101A3000E02AE182638380912402880F880F822B41
:101A40008483C5828E2D840F8195828380912402A8
:101A50008F5F8F738093240286E00F91EF90CF9079
:101A60000895FC0190818381808393839181292F44
:101A70002C7F84818370822B818384818C7F9370FF
:101A8000892B84838181846081839081890F8195F2
:101A900082830895CF93DF93EC01809128028823FD
:101AA000A1F18E81882389F5809186038093A60316
:101AB000809187038093A703809188038093A80374
:101AC000809189038093A90380918A038093AA035C
:101AD00080918B038093AB0386EA93E00E94310DE3
:101AE00020E030E0F901EA55FC4FDE01A20FB31F00
:101AF00090818C91981749F42F5F3F4F2630310524
:101B000089F71092280280E001C08FEFDF91CF911A
:101B1000089580E090E0FC01EA55FC4F8083019637
:101B200080329105C1F70895FF920F931F93CF93D1
:101B3000DF93EC01F62E0E94E70C892B31F08091A7
:101B400025028F5F8093250239C21981169516955B
:101B500010FD05C04C2FA6EAB3E0FE0107C0CE0180
:101B60006F2D0E944A0D46C281918D938E2F841B4A
:101B70008F15D0F30D8186EA93E00E94310D1A3063
:101B8000E1F11B3038F4143009F4F6C0163009F0D6
:101B9000F5C107C01C3209F480C0103309F0EEC152
:101BA000F2C1013009F0EAC11092AC031092AD030A
:101BB00084E88093AE030093AF031092B00381E5F5
:101BC0008093B10389E28093B20388E78093B303E3
:101BD0008CE68093B4031092B50380EF8093B60334
:101BE0008BE08093B7031092B8031092B903109260
:101BF000BA031092BB0346E1E3C1013191F0023117
:101C0000D1F1003109F0BAC11092AC030E94630215
:101C10008093AD030E9463029093AE031092AF03D2
:101C200055C1988580E02F81022F10E0082B192BD9
:101C3000F9841092AC030E9463022F2D30E0801BC8
:101C4000910B8217930720F40E946302F82EF01A7A
:101C5000F092AD03D801AE5BBD4FEEEAF3E02F2D5D
:101C600030E02E0F3F1F02C08D918193E217F307E2
:101C7000D9F74F2D96C11F2D1A50788560E08F81BE
:101C800090E0682B792BCE010996412F0E946602C5
:101C90008093AC031093AD038BC1073001F1083082
:101CA00078F4043009F446C0053018F4002309F133
:101CB00061C0053009F44DC0063009F05BC04EC06C
:101CC0000D3009F451C00E3020F4083009F052C034
:101CD0003AC00931C1F00A3109F04CC019C0109264
:101CE000AC031092AD03888569854A850E9468021D
:101CF0005FC11092AC031092AD0384E18093AE03F8
:101D00001092AF03FBC08F816B850E94C5024CC14E
:101D10008F816EEA73E00E94D402282F8F3F19F062
:101D20001092AC0303C089EC8093AC031092AD0316
:101D3000422F37C188850E948001882309F033C172
:101D40001092AC0333C188856EEA73E00E94800272
:101D500021C18EEA93E00E94A5021CC188856EEA2B
:101D600073E00E94AB0216C18F816EEA73E00E949D
:101D7000C70210C181EC18C1023209F470C00332ED
:101D800060F4013009F4EEC0013008F4D9C000322B
:101D9000A1F0013209F0F2C017C0073209F4BAC04D
:101DA000083220F4063209F0E9C0C1C00D3209F44E
:101DB00072C00F3209F0E2C0A7C01092AC0385E0F8
:101DC0008093AD0381E0D6C0688539857A852B85FF
:101DD000422F50E04831510514F08AECD0C0932FC7
:101DE00080E0E62FF0E0E82BF92BE630F10508F073
:101DF00089C0203408F086C0072F10E00034110598
:101E000008F080C01092AC03E530F10539F08E2F58
:101E10008F5F8093AD031092AE0305C08FEF809368
:101E2000AD038093AE034731510509F426E190E0FC
:101E3000EF01CC0FDD1FCA55DE4F0CC0F0E0EA55B4
:101E4000FC4FA881B981A00FB11F8C9180839F5F47
:101E50000F5F1F4FE92FE75F921780F3ABC08091B0
:101E600026029091270201969093270280932602E2
:101E7000892B31F481E090E0909327028093260231
:101E80001092AC0380912602909127028093AD03BB
:101E90009093AE0371C01092AC038E810E94A40196
:101EA0008430B1F0853020F48150823058F510C074
:101EB000803CD9F0823F31F51092AD0380EC8093E5
:101EC000AE038E810E94AF018093AF034AE078C0D9
:101ED0008E810E94AF018093AD0380EC8093AE03AE
:101EE0008E810E944002806C07C01092AD038093E7
:101EF000AE038E810E94AF018093AF031092B003B6
:101F00004BE05EC089EC3BC08E816DEA73E00E94BD
:101F1000890105C08E816DEA73E00E94B5018F3F93
:101F200009F441C01092AC03482F495F45C010929C
:101F3000AC038E816F812896AE010E94E50121C01D
:101F40008E818F3F19F41092D40106C081E08093F6
:101F5000D4018E818093D3018F81809323021092CC
:101F6000AC030FC01092AC038091D3018093AD03FA
:101F7000809123028093AE0349E022C081EC8093DC
:101F8000AC0347E01DC02896802FBE014EEA53E007
:101F90000E94D6028F3F39F01092AC031092AD032D
:101FA000482F485F09C089EC8093AC031092AD03C1
:101FB00048E006C0422F475F442311F48FEF1AC058
:101FC000942F20E007C09150E92FF0E0EA55FC4F34
:101FD0008081280F9923B9F7E42FF0E0EA55FC4FF0
:101FE000219520834F5F8091A60366EA73E00E94EB
:101FF000090380E0DF91CF911F910F91FF90089529
:1020000080912802882379F08091D401882311F4EB
:1020100081E008958091D30166E873E04091290240
:102020000E94090381E00895CF92EF92FF920F93EF
:102030001F93282F162FF42E86E893E0622F4091ED
:10204000D30120E000E074E0E72E52E0C52E0E94AC
:10205000110DE82FF0E0EA57FC4F94E090838F5F7A
:10206000E82FF0E0EA57FC4F91E090838F5FE82F74
:10207000F0E0EA57FC4F10838F5FE82FF0E0EA575B
:10208000FC4F90838F5FE82FF0E0EA57FC4FF0821F
:102090008F5FE82FF0E0EA57FC4F9FEF90838F5F50
:1020A000E82FF0E0EA57FC4F9083482F4F5F942FC2
:1020B00020E007C09150E92FF0E0EA57FC4F808103
:1020C000280F9923B9F7E42FF0E0EA57FC4F219548
:1020D00020834F5F4093290281E080932802809102
:1020E000D401882331F08091D30166E873E00E9427
:1020F00009031F910F91FF90EF90CF900895CF9219
:10210000EF92FF920F931F93282F162FF42E86E83D
:1021100093E0622F4091D30120E000E0F4E0EF2E45
:10212000E2E0CE2E0E94110DE82FF0E0EA57FC4FBE
:1021300094E090838F5FE82FF0E0EA57FC4F92EF36
:1021400090838F5FE82FF0E0EA57FC4F10838F5F9A
:10215000E82FF0E0EA57FC4F9FE690838F5FE82F6F
:10216000F0E0EA57FC4FF0828F5FE82FF0E0EA578B
:10217000FC4F9FEF90838F5FE82FF0E0EA57FC4F12
:102180009083482F4F5F942F20E007C09150E92F94
:10219000F0E0EA57FC4F8081280F9923B9F7E42F2C
:1021A000F0E0EA57FC4F219520834F5F40932902CE
:1021B00081E0809328028091D401882331F08091BE
:1021C000D30166E873E00E9409031F910F91FF900D
:1021D000EF90CF9008959FB7F894882311F4A298B8
:1021E000AA9A9FBF08959FB7F894882311F4A29AE2
:1021F000AA989FBF08959FB7F894882311F4A398D5
:10220000AB9A9FBF08959FB7F894882311F4A39ABF
:10221000AB989FBF0895DF93CF930F92CDB7DEB7F2
:102220008AE089838981815089838F5FD9F70F90F4
:10223000CF91DF910895DF93CF930F92CDB7DEB7A3
:10224000982F8FB7F894992311F4A398AB9A8FBF66
:102250008AE089838981815089838F5FD9F78FB71D
:10226000F894992311F4A298AA9A8FBF8AE08983DF
:102270008981815089838F5FD9F78FB7F89499232B
:1022800011F4A39AAB988FBF8AE08983898181502A
:1022900089838F5FD9F78FB7F894992311F4A29AA5
:1022A000AA988FBF8AE089838981815089838F5F53
:1022B000D9F70F90CF91DF910895DF93CF930F92CD
:1022C000CDB7DEB7982F8FB7F894992311F4A39A5E
:1022D000AB988FBF8AE089838981815089838F5F22
:1022E000D9F78FB7F894992311F4A298AA9A8FBFBF
:1022F0008AE089838981815089838F5FD9F78FB77D
:10230000F894992311F4A398AB9A8FBF8AE089833C
:102310008981815089838F5FD9F70F90CF91DF91A9
:102320000895DF93CF930F92CDB7DEB7982F8FB775
:10233000F894992311F4A39AAB988FBF8AE089830C
:102340008981815089838F5FD9F78FB7F89499235A
:1023500011F4A298AA9A8FBF8AE08983898181505B
:1023600089838F5FD9F78FB7F894992311F4A29AD4
:10237000AA988FBF8AE089838981815089838F5F82
:10238000D9F70F90CF91DF910895DF93CF930F92FC
:10239000CDB7DEB7982F8FB7F894992311F4A3988F
:1023A000AB9A8FBF8AE089838981815089838F5F4F
:1023B000D9F78FB7F894992311F4A298AA9A8FBFEE
:1023C0008AE089838981815089838F5FD9F78FB7AC
:1023D000F894992311F4A29AAA988FBF8AE089836E
:1023E0008981815089838F5FD9F70F90CF91DF91D9
:1023F0000895DF93CF930F92CDB7DEB7982F20E0EB
:102400003AE08FB7F894992311F4A29AAA988FBF53
:1024100067FF07C08FB7F894992349F4A398AB9A44
:1024200006C08FB7F894992311F4A39AAB988FBF85
:1024300039838981815089838F5FD9F78FB7F89469
:10244000992311F4A298AA9A8FBF39838981815068
:1024500089838F5FD9F72F5F283011F0660FD1CFB6
:102460008FB7F894992311F4A29AAA988FBF8FB7C7
:10247000F894992311F4A398AB9A8FBF8AE08983CB
:102480008981815089838F5FD9F78FB7F894992319
:1024900011F4A298AA9A8FBF8AE08983898181501A
:1024A00089838F5FD9F79923F1F494E62AE007C076
:1024B00029838981815089838F5FD9F791509B9BB4
:1024C00002C09923A9F79B9B09C0992339F48FB7C0
:1024D000F894A298AA9A8FBF9FEF06C08FB7F8947E
:1024E000A29AAA988FBF90E08AE08983898181505F
:1024F00089838F5FD9F7892F0F90CF91DF9108954E
:10250000DF93CF930F92CDB7DEB7382F8FB7F89404
:10251000332311F4A29AAA988FBF8FB7F89433236C
:1025200011F4A398AB9A8FBF8AE089838981815087
:1025300089838F5FD9F790E020E04AE0990F8FB749
:10254000F894332311F4A298AA9A8FBF4983898102
:10255000815089838F5FD9F7332311F49B99916060
:102560008FB7F894332311F4A29AAA988FBF4983A6
:102570008981815089838F5FD9F72F5F2830F1F6E9
:10258000892F0F90CF91DF910895DF93CF930F9212
:10259000CDB7DEB710922A029FB7F894882311F4C2
:1025A000A298AA9A9FBF9FB7F894882311F4A39882
:1025B000AB9A9FBF8AE089838981815089838F5F2D
:1025C000D9F78AE089838981815089838F5FD9F720
:1025D0008AE089838981815089838F5FD9F78AE076
:1025E00089838981815089838F5FD9F70F90CF913B
:1025F000DF910895DF93CF930F92CDB7DEB7982F79
:102600008AE089838981815089838F5FD9F78AE045
:1026100089838981815089838F5FD9F78AE0898393
:102620008981815089838F5FD9F78AE08983898185
:10263000815089838F5FD9F78FB7F894992311F46C
:10264000A298AA9A8FBF8FB7F894992311F4A398F0
:10265000AB9A8FBF10922A020F90CF91DF9108950D
:1026600080912A02089580932A020895DF92EF92C2
:10267000FF920F931F93CF93DF93F82E162FE72E21
:10268000D42E00912A020D7F016000932A020E943D
:102690001B11212F3E2DC901EC0110E00BC08F2D25
:1026A00069910E94F911882321F0006100932A02A8
:1026B00003C01F5F1D1598F38F2D0E945D1180913F
:1026C0002A028E7F826080932A02812FDF91CF9130
:1026D0001F910F91FF90EF90DF900895CF92DF92BE
:1026E000EF92FF920F931F93CF93DF93E82EEB01AE
:1026F000C42E10912A02177F84E0D82ED12AD092BE
:102700002A028E2D0E941B118E2D68810E94F911C4
:10271000882331F48E01FF24CC2DD0E0219719C0FD
:10272000146110932A02CC241FC08E2D0E948012A7
:10273000F80180838F2D90E08C179D0721F48E2D5A
:102740000E94C51103C08E2D0E949111F3940F5F5A
:102750001F4FFC1450F38E2D0E945D11FBEFDF2202
:1027600088E0D82AD0922A028C2DDF91CF911F9138
:102770000F91FF90EF90DF90CF900895AF92BF92AE
:10278000CF92DF92EF92FF920F931F93CF93DF933D
:10279000D82E5B01F42EC22E00912A02077F04601E
:1027A00000932A020E941B1110E0CF2DD0E0219748
:1027B00008C08D2DF70160810E94F9118823C9F4AA
:1027C0001F5F812F90E07501E80EF91E8C179D07A1
:1027D00084F38D2D0E941B118D2DF70160810E94C5
:1027E000F911882331F4750110E0CC2DD0E0219748
:1027F0001AC0006100932A02CC241EC08D2D0E94B5
:102800008012F7018083812F90E08C179D0721F4BF
:102810008D2D0E94C51103C08D2D0E9491111F5F47
:102820000894E11CF11C1C1548F38D2D0E945D11CC
:102830000B7F086000932A028C2DDF91CF911F91AE
:102840000F91FF90EF90DF90CF90BF90AF900895E1
:10285000DF93CF930F92CDB7DEB7198203C0898182
:102860008F5F89838981883CD0F30F90CF91DF916E
:102870000895DF93CF930F92CDB7DEB7482F20E0B6
:1028800030E00AC0198203C089818F5F8983898102
:10289000883CD0F32F5F3F4FE19B04C02F3F3105B1
:1028A00089F709C02F3F39F04EBB9FBB6DBBE29A41
:1028B000E19A80E001C08FEF0F90CF91DF910895F2
:1028C000DF93CF930F92CDB7DEB7482FFB0120E007
:1028D00030E00AC0198203C089818F5F89838981B2
:1028E000883CD0F32F5F3F4FE19B04C02F3F310561
:1028F00089F709C02F3F39F04EBB9FBBE09A8DB3DB
:10290000808380E001C08FEF0F90CF91DF91089519
:10291000DF92EF92FF920F931F93CF93DF937C018F
:10292000D42E8B01C0E0D0E00DC0CE018E0D9F1DD6
:10293000F80161918F010E9439142196882311F0CA
:102940008FEF03C0CD1588F380E0DF91CF911F9109
:102950000F91FF90EF90DF900895DF92EF92FF923A
:102960000F931F93CF93DF938C017B01D42EC0E094
:10297000D0E00DC0B7016C0F7D1FC8010E9460142C
:1029800021960F5F1F4F882311F08FEF03C0CD15E5
:1029900088F380E0DF91CF911F910F91FF90EF902E
:1029A000DF900895A1E21A2EAA1BBB1BFD010DC0EA
:1029B000AA1FBB1FEE1FFF1FA217B307E407F507EF
:1029C00020F0A21BB30BE40BF50B661F771F881FCB
:1029D000991F1A9469F760957095809590959B0161
:0C29E000AC01BD01CF010895F894FFCFB9
:1029EC001410010051120000000029640000C29A6A
:1029FC0000C94D43482D44544303005101000000CD
:102A0C0001C29A03480101800AA87A383880010073
:102A1C00000101002588000723280F7F80504B41BF
:102A2C00ECF6000202000000CA54656D7020436C85
:102A3C006F636B0300510100000002C29A00400258
:102A4C0001000000000000000400000101002588C6
:102A5C00E000780000FF0000847E006C7200000033
:102A6C000000CA56312E3220436C6F636B03005149
:102A7C000100000003C29A004002010000000000A7
:102A8C0000000400000101002588E000B40000FFF4
:102A9C000000C6BD00A2AB0000000000CA56312EDB
:102AAC003820436C6F636B0300510100000004C2BB
:102ABC009A00400201000000000000000400000D1C
:102ACC0001002588D000C00000FF0000D3CA00AD73
:102ADC00B60000000000CA56322E3520436C6F63DE
:102AEC006B0300510100000005C29A004002010076
:102AFC000000000000000400000D01002588D0003B
:102B0C00FD0000000000FFFF00E4F00000000000EA
:102B1C00CA56332E3320436C6F636BC082060000A1
:102B2C0000315A16000562007900B300ED00270150
:102B3C006101173A3A3A3A3A426F73746F6E205504
:102B4C006E6976657273697479004454430030423F
:062B5C00463000200100DC
:00000001FF
